:100000000C9421110C9452110C9452110C94521115
:100010000C9452110C9452110C9452110C945211D4
:100020000C9452110C9452110C9452110C945211C4
:100030000C9452110C9452110C9452110C945211B4
:100040000C9452110C94254B0C9452110C94521197
:100050000C9452110C9452110C9463BD0C9456BC28
:100060000C9452110C9429DC0C9452110C945211E2
:100070000C9452110C9452110C9452110C94521174
:100080000C942C530C9452110C9452110C94521148
:100090000C9452110C9452110C9452110C94521154
:1000A0000C9452110C9452110C94FE520C94521157
:1000B0000C9452110C9452110C9452110C94D05275
:1000C0000C9452110C9452110C9452110C9483BA4A
:1000D0000C945ABA0C9452110C9452110C94521163
:1000E0000C945211BB2CB42EED30942FC449C4494A
:1000F00026348E34DA34C449C4491737BB39893AB7
:10010000C449BA3CC449C4490F3EC449C4494841E2
:10011000C741394408469746F8B9FBB9EAB9EEB980
:10012000F4B932BAFFB903BA09BA0DBA11BA17BA9B
:100130001BBA1FBA32BA25BA29BA2DBA72BB77BB1D
:100140007CBB86BB90BB09BC9ABBA2BBAABBB4BBA1
:10015000BEBBC8BBD7BBE1BB09BCEBBBF5BBFFBBA0
:10016000084AD73B3BCE016E84BCBFFDC12F3D6C1E
:1001700074319ABD56833DDA3D00C77F11BED9E484
:10018000BB4C3E916BAAAABE000000803F05A84C64
:10019000CDB2D44EB93836A9020C50B99186880830
:1001A0003CA6AAAA2ABE000000803F004E414E494C
:1001B0004E495459494E46CDCCCC3D0AD7233C1725
:1001C000B7D13877CC2B329595E6241FB14F0A0072
:1001D0000020410000C84200401C4620BCBE4CCA62
:1001E0001B0E5AAEC59D7400407A10F35A00A072DF
:1001F0004E18090010A5D4E80000E8764817000062
:10020000E40B54020000CA9A3B000000E1F505002F
:100210000080969800000040420F000000A0860178
:10022000000000102700000000E803000000006448
:1002300000000000000A00000000000100000000B3
:10024000002C76D888DC674F0823DFC1DFAE59E188
:10025000B1B796E5E3E453C63AE651997696E8E6F7
:10026000C28426EB898C9B62ED407C6FFCEFBC9CCA
:100270009F40F2BAA56FA5F490055A2AF75C936BDC
:100280006CF9676DC11BFCE0E40D47FEF520E6B597
:1002900000D0ED902E0300943577050080841E0871
:1002A0000000204E0A000000C80C333333330F988F
:1002B0006E12831141EF8D2114893BE65516CFFE56
:1002C000E6DB18D1844B381BF77C1D901DA4BBE4E2
:1002D00024203284725E228100C9F124ECA1E53D24
:1002E00027434F4D4D554E49434154494F4E0044CD
:1002F000525952554E004552524F525300494E46A4
:100300004F004543484F0047322F47332062616416
:1003100020706172616D65746572730A005A207095
:10032000726F6265206F75742E206265640A0047E3
:100330003238205A20466F7262696464656E0A0022
:1003400047323900205A3A200020593A20004265AD
:100350006420583A20004D65736820706F696E7490
:100360002063616E6E6F74206265207265736F6CBE
:100370007665640A00456E642066696C65206C6968
:1003800073740A00426567696E2066696C65206C4B
:100390006973740A002E0A0046696C652862696EEA
:1003A000292064656C657465640044656C657469D6
:1003B0006F6E2862696E29206661696C65640053FE
:1003C00044207072696E74696E672062797465206A
:1003D000004E6F74205344207072696E74696E67AA
:1003E0000A002569730025696D2025697300256958
:1003F000682025696D2025697300256964202569B9
:10040000682025696D202569730025697920256993
:1004100064202569682025696D2025697300507264
:10042000696E742074696D653A200050726F74654E
:10043000637465642050696E0A000203FD02F602CF
:10044000EF02E1026F66660044454255473A004BB1
:10045000494C4C45442E20004D3131332053006F20
:100460006B002F2F200053657474696E67205472DF
:100470006176656C20416363656C65726174696F58
:100480006E3A200053657474696E67205265747209
:1004900061637420416363656C65726174696F6E3A
:1004A0003A200053657474696E67205072696E74E7
:1004B00020416363656C65726174696F6E3A2000F8
:1004C00053657474696E67205072696E7420616E32
:1004D000642054726176656C20416363656C65725B
:1004E0006174696F6E3A20000001363726FF033CC5
:1004F0003D38FF0E2E303E12FFFF0C0809FFFFFFB4
:100500001A1C18FFFF08440AFF43FFFFFFFFFFFF0D
:10051000206F7574206F662072616E67650A0053E4
:100520006572766F20003A200020536572766F2046
:100530000043290A0061626C656420286D696E20A1
:1005400074656D702000436F6C64206578747275FB
:10055000646573206172652000546F6F206661725C
:100560002066726F6D207265666572656E636520C8
:10057000706F696E740A00207A70726F62655F7ABC
:100580006F66667365743D20007A5F6D696E3A2010
:10059000202D3230207A5F6D61783A202032300091
:1005A0005A204F666673657420004E6F2063617336
:1005B00065206C696768740A004163746976652018
:1005C00045787472756465723A2000556E6B6E6F73
:1005D000776E20636F6D6D616E643A2022004D323C
:1005E00034004D3233202573004D313036205332E4
:1005F0003535004D31303920532569004D313930C2
:1006000020532569004739322045257300473020A3
:100610005A2573004D31303920532569004D313949
:100620003020532569004D323400473238004D34B4
:100630003230205330004D343230205331004731B6
:100640002046313030205A30004731205835302094
:100650005933303020463336303000473120463170
:100660003030205A330047312046313030205A3064
:100670000047312058333030205933303020463352
:100680003630300047312046313030205A33004771
:10069000312046313030205A300047312058333035
:1006A000302059353020463336303000473120462F
:1006B000313030205A330047312046313030205A13
:1006C00030004731205835302059353020463336F8
:1006D00030300047312046313030205A3300473126
:1006E0002046313030205A300047312058313830E0
:1006F00020593138302046333630300047312046DB
:10070000313030205A330047323900473930004702
:10071000323800473238205A3000473238004D38DE
:10072000340047312046323030205A302E300047D6
:1007300032380047393220452573004730205A258A
:1007400073004D31303920532569004D3139302047
:10075000532569004732382058302059300047323D
:1007600038205830205930004D3432302053310079
:100770004D343230205330002020506C616E6E6555
:100780007242756666657242797465733A2000201C
:1007900046726565204D656D6F72793A2000436F32
:1007A0006D70696C65643A20536570202034203286
:1007B0003031390A00207C20417574686F723A200C
:1007C000456E6465722D3520506C75730A003230A9
:1007D00031392D30392D303400204C61737420555F
:1007E0007064617465643A200056657220312E375A
:1007F000302E3120424C0A004D61726C696E00202F
:10080000536F6674776172652052657365740A0070
:10081000205761746368646F672052657365740A5A
:10082000002042726F776E206F7574205265736579
:10083000740A002045787465726E616C205265738D
:1008400065740A00506F77657255700A00737461A1
:1008500072740A006572726F722077726974696EC1
:100860006720746F2066696C650A00205A3A002080
:10087000593A0020583A00656E6473746F707320A3
:100880006869743A2000446F6E6520736176696E02
:10089000672066696C652E0A004D32390024F4D455
:1008A0003050C38E20C2A24017828B7011127A91F1
:1008B0000D816CD90AA861E108C7586607615143E8
:1008C000061E4B5D05C145A7041A411104093D9858
:1008D00003713931034036DB0265339102D4305461
:1008E00002802E1D02632CEE01752AC501B028A0DE
:1008F00001102781018F2564012B244B01E0223454
:1009000001AC211F018D200D01801FFC00841EED14
:1009100000971DDF00B81CD200E61BC600201BBCE0
:1009200000641AB200B219A8000A19A0006A189946
:1009300000D117910040178B00B516840031167E48
:1009400000B31579003A157300C7146F0058146A84
:1009500000EE1366008813630025135E00C7125B68
:10096000006C12570015125400C111510070114F44
:100970000021114B00D61049008D1047004610444D
:100980000002104200C00F4000800F3E00420F3CAA
:1009900000060F3B00CB0E3800930E37005C0E357F
:1009A00000270E3400F30D3200C10D3100900D30E0
:1009B00000600D2E00320D2D00050D2C00D90C2BE2
:1009C00000AE0C2900850C29005C0C2700350C2793
:1009D000000E0C2600E80B2400C40B2400A00B23FF
:1009E000007D0B23005A0B2100390B2100180B202E
:1009F00000F80A1F00D90A1E00BB0A1E009D0A1D2E
:100A000000800A1D00630A1C00470A1B002C0A1BF9
:100A100000110A1A00F7091A00DD091900C40919A2
:100A200000AB091900920917007B09180063091728
:100A3000004C09160036091600200916000A09158F
:100A400000F5081500E0081400CC081400B80814DC
:100A500000A4081400900813007D0812006B08130E
:100A6000005808120046081200340811002308112B
:100A7000001208110001081100F0071000E0071033
:100A800000D0071000C0071000B0070F00A107102A
:100A90000091070E0083070F0074070F0065070E13
:100AA0000057070E0049070E003B070D002E070EEA
:100AB0000020070D0013070D0006070D00F9060CB6
:100AC00000ED060D00E0060C00D4060C00C8060C74
:100AD00000BC060C00B0060C00A4060B0099060C26
:100AE000008D060B0082060B0077060B006C060BD0
:100AF0000061060A0057060B004C060A0042060A6F
:100B00000038060A002E060A0024060A001A060A01
:100B1000001006090007060A00FD050900F4050992
:100B200000EB050900E2050900D9050900D0050917
:100B300000C7050900BE050900B5050800AD050898
:100B400000A50509009C050800940508008C05080F
:100B500000840508007C050800740508006C050782
:100B600000650508005D050700560508004E0507ED
:100B70000047050700400508003805070031050754
:100B8000002A050700230507001C050600160507B7
:100B9000000F0507000805060002050700FB040614
:100BA00000F5040700EE040600E8040600E204076E
:100BB00000DB040600D5040600CF040600C90406C5
:100BC00000C3040600BD040600B7040600B1040516
:100BD00000AC040600A6040600A00405009B040661
:100BE0000095040500900406008A040500850405AC
:100BF00000800406007A04050075040500700405F1
:100C0000006B04050066040500610405005C040532
:100C10000057040500520405004D04050048040572
:100C200000430405003E0404003A040500350405B1
:100C300000300404002C04050027040400230405EC
:100C4000001E0404001A0404001604050011040424
:100C5000000D040400090405000404040000040459
:100C600000FC030400F8030400F4030400F0030490
:100C700000EC030400E8030400E4030400E00304C0
:100C800000DC030400D8030400D4030400D00304F0
:100C900000CC030400C8030300C503030024F404CC
:100CA000D9201BC40C5C0E9804C4095F026507714F
:100CB00001F405F900FB04B30048048700C103698F
:100CC000005803550003034500BE023A0084023178
:100CD0000053022A002902250004022000E4011C1E
:100CE00000C8011900AF0117009801140084011316
:100CF00000710110006101100051010E0043010D4F
:100D00000036010B002B010B0020010B001501091F
:100D1000000C01090003010800FB000800F30008B3
:100D200000EB000700E4000600DE000600D8000625
:100D300000D2000600CC000500C7000500C2000577
:100D400000BD000400B9000400B5000400B10004B7
:100D500000AD000400A9000400A5000300A20003E8
:100D6000009F0004009B0003009800030095000210
:100D70000093000300900003008D0002008B00032D
:100D80000088000200860002008400030081000247
:100D9000007F0002007D0002007B0002007900025B
:100DA000007700010076000200740002007200016A
:100DB00000710002006F0002006D0001006C000273
:100DC000006A00010069000200670001006600017E
:100DD0000065000100640002006200010061000182
:100DE00000600001005F0002005D0001005C000186
:100DF000005B0001005A0001005900010058000189
:100E00000057000100560001005500010054000188
:100E10000053000000530001005200010051000186
:100E200000500001004F0001004E0000004E000184
:100E3000004D0001004C0001004B0000004B000180
:100E4000004A00010049000100480000004800017C
:100E50000047000100460000004600010045000078
:100E60000045000100440001004300000043000170
:100E7000004200000042000100410000004100016A
:100E800000400001003F0000003F0001003E000064
:100E9000003E0001003D0000003D0001003C00005C
:100EA000003C0000003C0001003B0000003B000152
:100EB000003A0000003A000100390000003900014A
:100EC0000038000000380000003800010037000042
:100ED0000037000100360000003600000036000137
:100EE000003500000035000000350001003400002E
:100EF0000034000000340001003300000033000023
:100F00000033000100320000003200000032000116
:100F1000003100000031000000310001003000000D
:100F20000030000000300001002F0000002F000002
:100F3000002F0000002F0001002E0000002E0000F6
:100F4000002E0001002D0000002D0000002D0000EB
:100F5000002D0001002C0000002C0000002C0000DF
:100F6000002C0001002B0000002B0000002B0000D3
:100F7000002B0001002A0000002A0000002A0000C7
:100F8000002A0001002900000029000000290000BB
:100F900000290000002900010028000000280000AE
:100FA00000280000002800000028000100270000A1
:100FB0000027000000270000002700000027000194
:100FC0000026000000260000002600000026000089
:100FD000002600010025000000250000002500007B
:100FE000002500000025000000250001002400006D
:100FF0000024000000240000002400000024000160
:101000000023000000230000002300000023000054
:101010000023000000230000002300010022000044
:101020000022000000220000002200000022000038
:10103000002200010021000000210000002100002A
:10104000002100000021000000210000002100011B
:101050000020000000200000002000000020000010
:1010600000200000002000000020000000200001FF
:10107000001F0000001F0000001F0000001F0000F4
:10108000001F0000001F0000001F0001001E0000E4
:10109000001E0000001E0000001E0000004D38343D
:1010A00020582059205A20450047302046333630FA
:1010B00030205831383020593138300042696C695D
:1010C0006E656172204C6576656C696E672047724B
:1010D00069643A0A0020706F736974696F6E206FDB
:1010E0007574206F662072616E67652E0A003F502E
:1010F000726F626520002066697273740A005A007C
:1011000059005800486F6D65200052756E6E696E0B
:101110006720696E204452592D52554E206D6F64E0
:10112000650A00473239204175746F20426564209A
:101130004C6576656C696E670A0028422961636BAD
:1011400000284629726F6E740028522969676874F6
:1011500000284C29656674003F2856296572626F25
:101160007365206C6576656C20697320696D706CA1
:1011700061757369626C652028302D34292E0A0050
:10118000426164205A2076616C75650A004E6F20BA
:1011900062696C696E65617220677269640A0046F3
:1011A000696C652064656C657465643A0044656CBF
:1011B0006574696F6E206661696C65642C20466990
:1011C0006C653A20006F70656E206661696C6564BD
:1011D0002C2046696C653A2000202F002042403ABE
:1011E0000020403A00473238205830205930002043
:1011F000573A004732382058302059300020573AAB
:1012000000205A3A0020593A0020436F756E74202E
:10121000583A0020453A00205A3A0020593A0058DE
:101220003A002E0A006F70656E206661696C656415
:101230002C2046696C653A200057726974696E67A4
:1012400020746F2066696C653A2000534420636106
:101250007264206F6B0A006F70656E526F6F74203E
:101260006661696C65640A00766F6C756D652E69E0
:101270006E6974206661696C65640A004572726FFC
:10128000723A00534420696E6974206661696C0A81
:10129000004D3234004D3233202573006175746F78
:1012A00025692E6700656E7175657565696E6720C5
:1012B00022006563686F3A004B494C4C45442E2030
:1012C000005072696E7465722073746F707065641B
:1012D0002064756520746F206572726F72732E20A2
:1012E00046697820746865206572726F7220616E3D
:1012F0006420757365204D39393920746F2072650B
:1013000073746172742E202854656D7065726174F7
:101310007572652069732072657365742E2053653C
:1013200074206974206166746572207265737461DB
:101330007274696E67290A004E6F204C696E6520D1
:101340004E756D62657220776974682063686563A5
:101350006B73756D2C204C617374204C696E653A0B
:1013600020004E6F20436865636B73756D2077694D
:101370007468206C696E65206E756D6265722C20D4
:101380004C617374204C696E653A20006368656334
:101390006B73756D206D69736D617463682C204C7F
:1013A000617374204C696E653A20004C696E65204B
:1013B0004E756D626572206973206E6F74204C618A
:1013C0007374204C696E65204E756D6265722B31A9
:1013D0002C204C617374204C696E653A20004D31AD
:1013E0003130004D3331004D383420582059205AC7
:1013F00020450053442072656164206572726F72EB
:101400000A00446F6E65207072696E74696E6720A1
:1014100066696C650A0020496E76616C69642065B6
:10142000787472756465722000000000000000008E
:1014300000000000000000B4430000B4430000CDF1
:10144000435072696E7465722073746F7070656456
:101450002064756520746F206572726F72732E2020
:1014600046697820746865206572726F7220616EBB
:101470006420757365204D39393920746F20726589
:1014800073746172742E202854656D706572617476
:101490007572652069732072657365742E205365BB
:1014A000742069742061667465722072657374615A
:1014B0007274696E67290A0053544F502063616C3F
:1014C0006C65642062656361757365206F66204298
:1014D0004C546F756368206572726F72202D207294
:1014E0006573746172742077697468204D39393975
:1014F0000A0020746F6F206C6F6E672065787472BD
:101500007573696F6E2070726576656E7465640AB6
:101510000020636F6C6420657874727573696F6EF8
:101520002070726576656E7465640A0020204D38FF
:101530003531205A005A2D50726F6265204F666611
:1015400073657420286D6D293A0A002044002049F3
:101550000020204D33303120500050494420736525
:101560007474696E67733A0A00205A0020204D3463
:1015700032302053004175746F20426564204C6501
:1015800076656C696E673A0A00205A00205900207F
:10159000204D323036205800486F6D65206F6666EA
:1015A0007365743A0A00204500205A002059002033
:1015B000580020420020540020204D323035205366
:1015C00000416476616E6365643A20533C6D696ED8
:1015D0005F66656564726174653E20543C6D696E3A
:1015E0005F74726176656C5F66656564726174656F
:1015F0003E20423C6D696E5F7365676D656E745F1A
:1016000074696D655F6D733E20583C6D61785F78DD
:10161000795F6A65726B3E205A3C6D61785F7A5FD4
:101620006A65726B3E20453C6D61785F655F6A65F7
:10163000726B3E0A0020540020520020204D3230B0
:1016400034205000416363656C65726174696F6E2C
:101650002028756E6974732F7332293A20503C70BC
:1016600072696E745F616363656C3E20523C7265A3
:1016700074726163745F616363656C3E20543C7493
:10168000726176656C5F616363656C3E0A0020453C
:1016900000205A0020590020204D323031205800BF
:1016A0004D6178696D756D20416363656C6572612C
:1016B00074696F6E2028756E6974732F7332293ABE
:1016C0000A00204500205A0020590020204D3230C9
:1016D000332058004D6178696D756D2066656564CD
:1016E00072617465732028756E6974732F73293A5B
:1016F0000A00204500205A0020590020204D393290
:1017000020580053746570732070657220756E697F
:10171000743A0A0020204D3230302044300A002034
:10172000204D3230302044002044697361626C6582
:10173000640A0046696C616D656E7420736574742B
:10174000696E67733A0020204D3134392043203BC5
:1017500020556E69747320696E2043656C736975DA
:10176000730A002020473231202020203B20556E74
:1017700069747320696E206D6D0A007A5F6D696E01
:101780003A2000795F6D61783A2000785F6D61786A
:101790003A20005265706F7274696E6720656E64DE
:1017A00073746F70207374617475730A0043617091
:1017B0003A454D455247454E43595F504152534576
:1017C000523A300A004361703A434153455F4C49F5
:1017D0004748545F4252494748544E4553533A3064
:1017E0000A004361703A544F47474C455F4C4947A4
:1017F0004854533A300A004361703A534F465457A5
:101800004152455F504F5745523A300A004361708C
:101810003A4C4556454C494E475F444154413A3154
:101820000A004361703A5A5F50524F42453A310ABA
:10183000004361703A4155544F4C4556454C3A313E
:101840000A004361703A5052494E545F4A4F423A3F
:10185000310A004361703A50524F47524553533A50
:10186000300A004361703A4155544F5245504F522F
:10187000545F54454D503A310A004361703A454532
:1018800050524F4D3A310A004649524D5741524548
:101890005F4E414D453A4D61726C696E20566572DE
:1018A00020312E37302E3120424C20284372656182
:1018B0006C69747933442920534F555243455F4333
:1018C0004F44455F55524C3A68747470733A2F2FE9
:1018D0006769746875622E636F6D2F4D61726C69F4
:1018E0006E4669726D776172652F4D61726C696EBB
:1018F0002050524F544F434F4C5F56455253494F1F
:101900004E3A312E30204D414348494E455F54599F
:1019100050453A456E6465722D3520506C757320C4
:1019200045585452554445525F434F554E543A31F1
:1019300020555549443A63656465326132662D34F9
:101940003161322D343734382D396231322D6335DF
:10195000356336326633363766660A00205A002011
:101960005900580020204D61783A2000205A00206C
:101970005900580020204D696E3A20004F6E20001B
:101980004F666600536F667420656E6473746F7083
:10199000733A200020643A0020693A0020703A002F
:1019A00023646566696E65202044454641554C5464
:1019B0005F4B64200023646566696E6520204445A2
:1019C0004641554C545F4B69200023646566696E3F
:1019D00065202044454641554C545F4B70200050D3
:1019E0004944204175746F74756E652066696E692F
:1019F00073686564212050757420746865206C617B
:101A00007374204B702C204B6920616E64204B64F2
:101A100020636F6E7374616E74732066726F6D20D5
:101A200062656C6F7720696E746F20436F6E6669B4
:101A30006775726174696F6E2E680A0050494420A0
:101A40004175746F74756E65206661696C6564219B
:101A50002074696D656F75740A00504944204175A2
:101A6000746F74756E65206661696C6564212054BD
:101A7000656D706572617475726520746F6F206832
:101A80006967680A00204B643A2000204B693A20BD
:101A900000204B703A20000A20436C617373696325
:101AA00020504944200A002054753A2000204B75EC
:101AB0003A2000206D61783A2000206D696E3A204E
:101AC0000020643A200020626961733A20004F666A
:101AD000660A00466164652048656967687420008D
:101AE000426564204C6576656C696E6720004661CE
:101AF000696C656420746F20656E61626C6520425C
:101B00006564204C6576656C696E670A004D657387
:101B10006820706F696E742063616E6E6F742062EE
:101B200065207265736F6C7665640A004D343231DE
:101B300020696E636F727265637420706172616D8B
:101B4000657465722075736167650A00290A002053
:101B500062797465733B206372632000536574740B
:101B6000696E67732053746F7265642028002028A3
:101B700063616C63756C6174656429210A002021BE
:101B80003D2000454550524F4D20435243206D6942
:101B9000736D61746368202D202873746F7265649F
:101BA000292000290A002062797465733B20637242
:101BB0006320002073746F726564207365747469A8
:101BC0006E6773207265747269657665642028009B
:101BD000204D61726C696E3D563431290A002845EA
:101BE0004550524F4D3D00454550524F4D20766572
:101BF0007273696F6E206D69736D61746368200024
:101C000048617264636F6465642044656661756CE5
:101C1000742053657474696E6773204C6F616465DA
:101C2000640A00F4010000F401000064000000E810
:101C300003000000009643000096430000A040000F
:101C400000C8410000A0420000A04200004844003B
:101C500000BA4250726F62696E67206661696C6596
:101C6000640A00205A3A200020593A200042656454
:101C700020583A20005072696E7465722068616C59
:101C80007465642E206B696C6C28292063616C6C10
:101C90006564210A000000B4430000B44300000062
:101CA0000000004842000048420000804000000060
:101CB000005761726E696E673A20486F6D696E6792
:101CC0002042756D702044697669736F72203C20E4
:101CD000310A000202040000A0400000A040000001
:101CE00000400000B4430000B4430000CD430101B4
:101CF000FF62696E004D31313720494E56414C49E3
:101D00004420444154412E00473932205A25732043
:101D10004525730062696E00526573656E643A20F2
:101D2000006F6B0020746F6F206C6F6E672065789A
:101D300074727573696F6E2070726576656E746506
:101D4000640A0020636F6C6420657874727573692F
:101D50006F6E2070726576656E7465640A006275D8
:101D600073793A2070617573656420666F722069BB
:101D70006E7075740A00627573793A2070617573BC
:101D8000656420666F7220757365720A00627573F0
:101D9000793A2070726F63657373696E670A004BDE
:101DA000494C4C45442E20004B494C4C20636175F6
:101DB000736564206279204B494C4C2062757474C1
:101DC0006F6E2F70696E0A004B494C4C45442E20B3
:101DD000004B494C4C206361757365642062792027
:101DE000746F6F206D75636820696E6163746976C6
:101DF000652074696D65202D2063757272656E743F
:101E000020636F6D6D616E643A20007C3C3E5E2BFA
:101E10003D3F2F5B5D3B2C2A225C0070012C019022
:101E2000012701B0012201C0011D01F001180110BC
:101E300002130130020E016002090190020401C088
:101E400002FF000003FA004003F5008003F000D019
:101E500003EB002004E6007004E100E004DC004035
:101E600005D700C005D2004006CD00D006C80080CE
:101E700007C3003008BE00F008B900C009B400B0C4
:101E80000AAF00B00BAA00D00CA500000EA00050B5
:101E90000F9B00C01096005012910000148C00C0DF
:101EA000158700B0178200B0197D00D01B780000A4
:101EB0001E730040206E0090226900F024640040F0
:101EC000275F0090295A00E02B5500102E5000206B
:101ED000304B0010324600E033410090353C00109A
:101EE00037370070383200A0392D00B03A2800A0F2
:101EF0003B2300603C1E00103D1900903D14001073
:101F00003E0F00703E0A00C03E0500003F0000404A
:101F10003FFBFF803FF6FFC03FF1FF0000210024A0
:101F20000027002A002D00300033000101000004CA
:101F30000107010A0100002200250028002B002EC5
:101F4000003100340002010000050108010B01000E
:101F50000020002300260029002C002F0032000062
:101F60000100000301060109010505050507050833
:101F7000080808020202020A0A080804040404010C
:101F8000010101010101010303030303030303042E
:101F90000707070C0C0C0C0C0C0C0C0202020206BE
:101FA000060606060606060B0B0B0B0B0B0B0B01AE
:101FB000021020200808102040102040800201025A
:101FC0000108040201010204081020408080402022
:101FD000100804020180040201804020100804025D
:101FE00001080402010102040810204080010204DB
:101FF000081020408000000A0B02090C0D0E080793
:1020000003040100000000000000000000000000C8
:1020100000000000000000000000000000000000C0
:10202000001211100000000000000000000000007D
:1020300000000000000000000000006265640A006B
:102040002C2073797374656D2073746F7070656480
:1020500021204865617465725F49443A20004572E9
:10206000723A204D415854454D5020424544004558
:1020700072723A204D415854454D50004D415854CC
:10208000454D5020747269676765726564004572DA
:10209000723A204D494E54454D502042454400452A
:1020A00072723A204D494E54454D50004D494E54A0
:1020B000454D5020747269676765726564004865B4
:1020C0006174696E67206661696C6564004865616A
:1020D00074696E67206661696C6564004865617447
:1020E000696E67206661696C656400486561746942
:1020F0006E67206661696C656400544845524D41C5
:102100004C2052554E4157415900546865726D61DB
:102110006C2052756E617761790057726974696ECF
:102120006720746F2066696C653A20006F70656E79
:10213000206661696C65642C2046696C653A2000F4
:102140006F70656E206661696C65642C2046696CF1
:10215000653A200046696C652073656C656374653B
:10216000640A002053697A653A200046696C65204C
:102170006F70656E65643A20006F70656E206661F1
:10218000696C65642C2046696C653A20002066699C
:102190006C653A20004E6F7720002220706F73002C
:1021A0002220706172656E743A2200535542524F7C
:1021B0005554494E452043414C4C2074617267652B
:1021C000743A22004B494C4C45442E2000747279DD
:1021D000696E6720746F2063616C6C207375622D6B
:1021E00067636F64652066696C65732077697468DE
:1021F00020746F6F206D616E79206C6576656C73ED
:102200002E204D4158206C6576656C2069733A002C
:1022100043616E6E6F74206F70656E2073756264BB
:10222000697220004572726F722077726974696EEC
:102230006720746F20454550524F4D210A0074E6C7
:10224000B9E711241FBECFEFD1E2DEBFCDBF00E062
:102250000CBF15E0A0E0B2E0E2E0FEEE01E00BBF53
:1022600002C007900D92AE36B107D9F72CE1AEE669
:10227000B5E001C01D92A133B207E1F711E1C0E260
:10228000D1E100E006C021970109802FFE010E94E4
:102290003BF6CF31D10780E00807A9F70E9452DC56
:1022A0000C94F0F60C9400002F923F924F925F92A4
:1022B0006F927F928F929F92AF92BF92CF92DF9256
:1022C000EF92FF920F931F93CF93DF93CDB7DEB7BB
:1022D000CF55D1090FB6F894DEBF0FBECDBF009128
:1022E0003D1720E6029F800111240F5B194F80915A
:1022F000911680FF1AC0E2EBF2E184917F013FEF7B
:10230000E31AF30A811102C0780104C00E9414DBB1
:10231000F701F3CFD7018D917D01882319F00E9439
:1023200014DBF8CF8AE00E9414DB81E090E0909308
:10233000581B8093571B10929105109290058FE3C4
:1023400080939B0510929A051092990584E0E8E825
:10235000F5E0DF011D928A95E9F7F80180810F5FB2
:102360001F4F8032D1F38E34C9F4818190ED980FE4
:102370009A3020F08D3211F08B3281F4DF01129609
:102380009D012F5F3F4F8C9180538A3010F4D9010B
:10239000F7CFFD01119680818032D9F3F0935F1B56
:1023A000E0935E1B7F01BFEFEB1AFB0A10816AE22C
:1023B00070E0C7010E9489F6009731F0FC01319767
:1023C00080818032E1F311821D3431F1143521F125
:1023D000173411F1E2EBF2E184918F010F5F1F4F8F
:1023E000882321F00E9414DBF801F6CF60915E1B78
:1023F00070915F1B8BEC95E00E94AD5382E20E94CE
:1024000014DB8AE00E9414DB1092581B1092571BB9
:102410000E9480B10C94852AC701FC01208101969D
:102420002032D9F320532A30A8F610939B0580E080
:1024300090E06AE03196DF0111972C91022E000C9A
:10244000330B20533109689FA001699F500D11245F
:10245000C901840F951F208120532A3058F390938F
:102460009A0580939905DF0131962C912032D9F39A
:102470001D34D1F48E31910591F03CF487319105F2
:1024800071F08C31910581F40AC08537910564F0B3
:102490008737910524F0803AE3E09E0729F4B09352
:1024A0009105A09390057DC0109291051092900522
:1024B00000915E1BEE24E394F12CFD0131962C91EA
:1024C000222309F46EC02132A9F41D3499F480321C
:1024D000910581F4F0939105E093900563E270E03B
:1024E000CF010E9489F6009711F40C94951EDC012F
:1024F0001C9257C021542A31A0F5AF01FA01308156
:102500004F5F5F4F3032D1F340ED430F4A3040F020
:1025100043ED430F423020F03B3211F00C94AB29D5
:10252000AF01622F70E0DB0133E0B595A7953A95D6
:10253000E1F7A857BA4F2770670102C0CC0CDD1C29
:102540002A95E2F796013C91232B2C9341155105D6
:1025500011F0401B01C040E0DB01A259BA4F4C937F
:102560000AC02091900530919105232B21F4B0935E
:102570009105A0939005208121542A3110F4DF01A8
:102580009CCFDF01AD014F5F5F4F2C9120532A306C
:1025900010F4DA01F7CFFD01119620812032D9F332
:1025A000EECF80919B058D3411F40C94951E8435EB
:1025B00011F40C946A29873409F00CCF2090990506
:1025C00030909A052CE12216310409F485C694F462
:1025D00044E02416310444F452E0251631040CF092
:1025E000FEC037FE2FC010CF84E02816310409F456
:1025F0002EC60ACF9AE22916310411F40C94E31D79
:102600006CF4BDE12B16310411F40C94C01CEEE106
:102610002E16310411F40C94C41CF6CEFBE52F16D3
:10262000310411F40C94481D2CE52216310411F4E8
:102630000C944D1D3AE52316310409F0E5CE1092B5
:102640009805E2CE80916002882309F4DDCE0E94D5
:1026500082540E9442AE8091281C813021F482E095
:102660008093281CD1CE90917712992309F4CCCE77
:10267000823009F4C9CE8091220690912306893BCD
:102680009105DCF06091220670912306072E000C64
:10269000880B990B0E94A7EC9B01AC016091FC0593
:1026A0007091FD058091FE059091FF050E94A1ECBF
:1026B00087FF03C00E9450ABE5CF1092431781E023
:1026C00080933C0280EA9FE09093E81B8093E71B95
:1026D0008091261C882349F182E090E090937E153A
:1026E00080937D1585E08093711512E81093741521
:1026F00084E190E1A0E0B0E08093751590937615A9
:10270000A0937715B09378150E94566661E070E04B
:1027100080E090E00E9412BC81E09AE590937E15E3
:1027200080937D158BE090E028C08EE090E0909340
:102730007E1580937D1585E08093711512E81093C6
:10274000741584E190E1A0E0B0E08093751590935A
:102750007615A0937715B09378150E94566661E0C0
:1027600070E080E090E00E9412BC81E09AE59093D6
:102770007E1580937D1585E390E09093801580937E
:102780007F1587E0809371151093741584E890E0AD
:10279000A0E0B0E08093751590937615A09377151F
:1027A000B09378150E94566681E080934917809314
:1027B000281C8091C71A9091C81A019739F40E9479
:1027C0009E6A7093C81A6093C71A04C01092C81A00
:1027D0001092C71A1092C51A1092C61A15CE80917F
:1027E0006002882309F410CE0E94825482E50E9480
:1027F000F7DA882309F43CC10E9491DA4B015C01AD
:102800008091DC169091DD16A091DE16B091DF1656
:102810008CA79DA7AEA7BFA72091E0163091E11627
:102820004091E2165091E31628AB39AB4AAB5BAB53
:102830008091931A9091941AA091951AB091961A3A
:1028400088AF99AFAAAFBBAF2091971A3091981A71
:102850004091991A50919A1A2CAB3DAB4EAB5FAB9D
:1028600020E030E0A901C501B4010E94A1EC882359
:1028700009F42AC128AD39AD4AAD5BAD6CA57DA583
:102880008EA59FA50E94A1EC81110DC02CA93DA988
:102890004EA95FA968A979A98AA99BA90E94A1EC60
:1028A000882309F411C111E032E02316310409F044
:1028B00010E020E030E0A901C501B4010E94A1ECC4
:1028C000881F8827881F181759F080E090E0A0E83B
:1028D000BFEB28968CAF9DAFAEAFBFAF28970AC0B5
:1028E00020E030E040E85FE328962CAF3DAF4EAFEC
:1028F0005FAF28972CA53DA54EA55FA568AD79AD26
:102900008AAD9BAD0E943AF324966CAF7DAF8EAF3B
:102910009FAF249728A939A94AA95BA96CA97DA9C9
:102920008EA99FA90E943AF36B017C0124962CADDD
:102930003DAD4EAD5FAD2497CA01B9010E9406EDD1
:102940002B013C01A7019601C701B6010E9406EDCB
:102950009B01AC01C301B2010E943BF30E94A7F5A9
:102960006CAF7DAF8EAF9FAF20E030E040E05FE323
:102970000E9406ED2B013C01A5019401C501B401A3
:102980000E9406ED4B015C01A3019201C301B2015B
:102990000E9406ED9B01AC01C501B4010E943AF30F
:1029A0000E94A7F528962CAD3DAD4EAD5FAD2897A2
:1029B0000E9406ED4B015C01C701B60190582CAD99
:1029C0003DAD4EAD5FAD0E9417F4A50194010E948C
:1029D00006ED6B017C0128AD39AD4AAD5BAD6CA550
:1029E0007DA58EA59FA50E943BF320E030E040E04E
:1029F0005FE30E9406ED9B01AC01C701B6010E9496
:102A00003BF32CA53DA54EA55FA50E943AF36B01B3
:102A10007C012CA93DA94EA95FA968A979A98AA919
:102A20009BA90E943BF320E030E040E05FE30E947E
:102A300006ED2B013C012CAD3DAD4EAD5FAD2496B6
:102A40006CAD7DAD8EAD9FAD24970E9417F4A501AE
:102A500094010E9406ED9B01AC01C301B2010E94EA
:102A60003BF328A939A94AA95BA90E943AF314C0EB
:102A700089E40E94F7DA882329F00E9491DA6B0139
:102A80007C0103C0C12CD12C76018AE40E94F7DAC4
:102A90008823E9F00E9491DA68AF79AF8AAF9BAFE3
:102AA00020E030E0A901C701B6010E94A1EC81112C
:102AB0001BC020E030E0A90168AD79AD8AAD9BADC7
:102AC0000E94A1EC811110C0ECE7F2E1ADC320E05F
:102AD00030E0A901C701B6010E94A1EC8823A1F34F
:102AE00018AE19AE1AAE1BAED701C601B0588CA7EE
:102AF0009DA7AEA7BFA728AD39AD4AAD5BAD505875
:102B000028AB39AB4AAB5BAB9C01AD01BC01CD013D
:102B10000E9406ED4B015C0128A939A94AA95BA9CD
:102B2000CA01B9010E9406ED9B01AC01C501B401C7
:102B30000E943BF30E94A7F564966CAF7DAF8EAF09
:102B40009FAF64978091DC169091DD16A091DE1600
:102B5000B091DF168CAB9DABAEABBFAB9C01AD01B2
:102B6000C701B6010E943BF328966CAF7DAF8EAFD4
:102B70009FAF28972091E0163091E1164091E21620
:102B80005091E3162CAF3DAF4EAF5FAF28AD39ADDE
:102B90004AAD5BAD6CAD7DAD8EAD9FAD0E943BF39C
:102BA00068966CAF7DAF8EAF9FAF68978091931A98
:102BB0009091941AA091951AB091961A2C968CAF78
:102BC0009DAFAEAFBFAF2C9728962CAD3DAD4EADAF
:102BD0005FAD2897BC01CD010E943AF36B017C01E7
:102BE0002091971A3091981A4091991A50919A1AF7
:102BF00060962CAF3DAF4EAF5FAF609768962CAD3F
:102C00003DAD4EAD5FAD689760966CAD7DAD8EAD60
:102C10009FAD60970E943AF34B015C018091E416EE
:102C20009091E516A091E616B091E7166C968CAFE0
:102C30009DAFAEAFBFAF6C979C01AD0160919B1A89
:102C400070919C1A80919D1A90919E1A0E943AF35D
:102C500024966CAF7DAF8EAF9FAF2497A7019601EE
:102C60006CA57DA58EA59FA50E9406ED2B013C01BC
:102C7000A501940168A979A98AA99BA90E9406EDDA
:102C80009B01AC01C301B2010E943BF32B013C014B
:102C9000A50194016CA57DA58EA59FA50E9406EDBA
:102CA0004B015C01A701960168A979A98AA99BA992
:102CB0000E9406ED9B01AC01C501B4010E943AF3EC
:102CC000A30192010E94AEF36B017C0120E030E091
:102CD000A9010E94A1EC87FF0AC02BED3FE049EC5F
:102CE00050E4C701B6010E943BF36B017C0192E006
:102CF0002916310451F42BED3FE049EC50E4C701B3
:102D0000B6010E943AF36B017C0120E030E0A9019A
:102D1000C701B6010E94A1EC811124C02C962CADF4
:102D20003DAD4EAD5FAD2C976CA97DA98EA99FA935
:102D30000E94A1EC811116C060962CAD3DAD4EAD48
:102D40005FAD60976CAD7DAD8EAD9FAD0E94A1EC87
:102D5000811108C00BEDC02E0FE0D02E09ECE02E43
:102D600000E4F02EA701960164966CAD7DAD8EADAA
:102D70009FAD64970E9406ED9B01AC010E9406ED99
:102D80004B015C0124962CAD3DAD4EAD5FAD24975B
:102D9000CA01B9010E9406ED9B01AC01C501B40155
:102DA0000E943BF30E94A7F54B015C012FE632E144
:102DB00043E85AE30E94A1EC87FD30C2C501B4018B
:102DC0000E94B0F40E9484F47DAF6CAFDB01AB2BAA
:102DD00021F4E1E0F0E0FDAFECAF4090E816509058
:102DE000E9166090EA167090EB162CAD3DADB90176
:102DF00080E090E00E94A5EC4B015C019B01AC01DE
:102E0000C701B6010E9417F46CAB7DAB8EAB9FABD4
:102E1000A501940124966CAD7DAD8EAD9FAD249738
:102E20000E9417F464966CAF7DAF8EAF9FAF64972E
:102E3000A301920160919F1A7091A01A8091A11A2A
:102E40009091A21A0E943AF3A50194010E9417F4EE
:102E5000A0966CAF7DAF8EAF9FAFA0972CA93DA978
:102E60004EA95FA9CA01B9010E9406ED20E030E039
:102E700040E05FE30E9406ED9B01AC0160E070E082
:102E800080E89FE30E943AF324966CAF7DAF8EAF4B
:102E90009FAF24976C968CAD9DADAEADBFAD6C97DA
:102EA00089879A87AB87BC874D865E866F86788ACE
:102EB00060910B0270910C02072E000C880B990B8D
:102EC0000E94A7EC209134023091350240913602E5
:102ED000509137020E9406ED2AE037ED43E25CE3B1
:102EE0000E9406ED2C966CAF7DAF8EAF9FAF2C97F6
:102EF0000E944ABC9B01AC0128533F4F4F4F5F4F8C
:102F000060962CAF3DAF4EAF5FAF60974CA45DA411
:102F10006EA47FA422242394312C19E1D12E4CAD30
:102F20005DAD4215530509F435C10E9429CA0E94BE
:102F30004ABCDC01CB0160962CAD3DAD4EAD5FAD22
:102F40006097821B930BA40BB50BB7FD10C00E94BA
:102F50004ABC9B01AC0128533F4F4F4F5F4F6096D7
:102F60002CAF3DAF4EAF5FAF60970E9450ABDA948D
:102F7000DD2009F441C028A939A94AA95BA92496F2
:102F80006CAD7DAD8EAD9FAD24970E9406ED4B01DB
:102F90005C019201A3016CA97DA98EA99FA90E9441
:102FA00006EDA50194010E943BF37B018C01920187
:102FB000A30124966CAD7DAD8EAD9FAD24970E948C
:102FC00006ED4B015C0128A939A94AA95BA96CA9A6
:102FD0007DA98EA99FA90E9406ED9B01AC01C501A8
:102FE000B4010E943AF32B013C01C701D80188AB20
:102FF00099ABAAABBBAB4DC0B10180E090E00E94A1
:10300000A5EC2CA93DA94EA95FA90E9406ED4B0194
:103010005C010E9414F46B017C01C501B4010E94A3
:103020009DF54B015C01A70196016CA57DA58EA5C0
:103030009FA50E9406ED2B013C0128AD39AD4AAD9C
:103040005BADC501B4010E9406EDA30192010E948F
:103050003BF32B013C01A50194016CA57DA58EA538
:103060009FA50E9406ED4B015C0128AD39AD4AAD2C
:103070005BADC701B6010E9406ED9B01AC01C50125
:10308000B4010E943AF368AB79AB8AAB9BABA9E180
:10309000DA2E9201A30128966CAD7DAD8EAD9FAD69
:1030A00028970E943BF369837A838B839C8328A9AA
:1030B00039A94AA95BA968966CAD7DAD8EAD9FAD6F
:1030C00068970E943BF36D837E838F839887649615
:1030D0002CAD3DAD4EAD5FAD649769857A858B852E
:1030E0009C850E943BF369877A878B879C87A09693
:1030F0002CAD3DAD4EAD5FADA0976D857E858F85C6
:1031000098890E943BF36D877E878F87988B80918B
:103110003302882321F0CE0101960E94B0A7C0900F
:10312000930589819A81AB81BC8188A399A3AAA3C5
:10313000BBA38D819E81AF81B8858CA39DA3AEA3D7
:10314000BFA389859A85AB85BC8588A799A7AAA7BF
:10315000BBA7AE01485D5F4FBE016C5D7F4FCE01E6
:1031600080960E9436812C96ECACFDAC0EAD1FAD66
:103170002C979E01235F3F4FAE01485D5F4FBE011C
:103180006C5D7F4FCE0180960E941D743FEF231A25
:10319000330AC5CEC09093058091931A9091941AEA
:1031A000A091951AB091961A88A399A3AAA3BBA33C
:1031B0008091971A9091981AA091991AB0919A1AA1
:1031C0008CA39DA3AEA3BFA380919B1A90919C1A40
:1031D000A0919D1AB0919E1A88A799A7AAA7BBA7EC
:1031E000AE01485D5F4FBE016C5D7F4FCE018096A2
:1031F0000E9436812C96ECACFDAC0EAD1FAD2C9729
:103200002FE93AE1AE01485D5F4FBE016C5D7F4F33
:10321000CE0180960E941D740E94316E0E9409DBCF
:10322000F3C80E9414DBF80184918F010F5F1F4FD8
:103230008111F7CFE7E0F3E084918F010F5F1F4F1B
:10324000882309F4E1C80E9414DBF801F5CF80E57A
:103250000E94F7DA882379F080918C0590918D0592
:10326000009749F04AE050E060E070E00E9420EBF7
:103270006B017C0103C0C12CD12C760183E50E9437
:10328000F7DA882361F00E9491DA20E030E04AE723
:1032900054E40E9406ED0E9484F46B017C010E94BC
:1032A00029CE0E9409DB8091A31A9091A41AA091C3
:1032B000A51AB091A61AC80ED91EEA1EFB1E0E94BE
:1032C0004ABCDC01CB018C199D09AE09BF09B7FFCF
:1032D0009BC80E9450ABF3CF0E9429CE80E00E9491
:1032E000716B0E94336C11E01093F40588E50E9425
:1032F000C8DAE82E89E50E94C8DA082F8AE50E941C
:10330000C8DAF82EE11004C0011104C0182705C066
:10331000011102C010E001C0182F0E94276E111188
:1033200005C0E11003C0002309F440C020E030E0F4
:1033300040EA50E46091F4167091F5168091F6160B
:103340009091F7160E943BF360939B1A70939C1A1E
:1033500080939D1A90939E1A2091E4163091E51661
:103360004091E6165091E7160E9461F518165CF43C
:1033700019821A821B821C82BE016F5F7F4F8BE90C
:103380009AE10E94446D111105C0E11003C00111C2
:1033900007C00CC080E090E00E9473A61123B9F32F
:1033A00081E090E00E9473A6111103C0FF2009F490
:1033B000CEC08091F505882321F08091F60581111A
:1033C0001AC0E2EBF2E184918F010F5F1F4F811170
:1033D00003C0EFE2F3E004C00E9414DBF801F3CF76
:1033E00084918F010F5F1F4F882309F4B0C00E94A2
:1033F00014DBF801F5CF0E941ADA4090EC165090D9
:10340000ED166090EE167090EF1620E030E044E389
:1034100053E4C301B2010E943BF34B015C01609392
:10342000931A7093941A8093951A9093961A809198
:10343000F0169091F116A091F216B091F3168CA7A8
:103440009DA7AEA7BFA720E030E044E353E4BC0152
:10345000CD010E943BF36B017C016093971A70933E
:10346000981A8093991A90939A1A8091E4169091E1
:10347000E516A091E616B091E71680939B1A9093FB
:103480009C1AA0939D1AB0939E1AA3019201C501A4
:10349000B4010E943AF34B015C012FE632E143E8AC
:1034A0005AEB0E9461F587FD0AC021E230E044EB4F
:1034B00053E4C501B4010E94A1EC18161CF4E2EB20
:1034C000F2E133C02CA53DA54EA55FA5C701B6010D
:1034D0000E943AF36B017C012FE632E143E85AEB9C
:1034E0000E9461F587FDEBCF21E230E044EB53E42D
:1034F000C701B6010E94A1EC18160CF319821A82BA
:103500001B821C829E012F5F3F4F44EE56E167E90C
:103510007AE183E99AE10E94536C82E090E00E9494
:1035200073A615C00E9414DBF80184918F010F5F10
:103530001F4F8111F7CFEDE1F3E084918F010F5F11
:103540001F4F882321F00E9414DBF801F6CF0E9460
:103550001ADA80912A1C813009F059C080933C020C
:1035600080E090E00E94C2BC8091261C882319F163
:1035700084E090E090937E1580937D1585E08093A4
:10358000711512E81093741584E190E1A0E0B0E0A9
:103590008093751590937615A0937715B093781551
:1035A0000E94566681E09AE590937E1580937D1582
:1035B0008CE090E022C080E190E090937E158093B3
:1035C0007D1585E08093711512E81093741584E1E0
:1035D00090E1A0E0B0E08093751590937615A093EC
:1035E0007715B09378150E94566681E09AE590931E
:1035F0007E1580937D1586E390E0909380158093EF
:103600007F1587E080937115109374152AC085305B
:10361000B1F581E080933C0280E090E00E94C2BC62
:1036200010922A1C8091261C882349F081E09AE59B
:1036300090937E1580937D158CE290E008C081E028
:103640009AE590937E1580937D1581E590E09093A7
:10365000801580937F1587E08093711582E88093B1
:10366000741584E890E0A0E0B0E080937515909325
:103670007615A0937715B09378150E9456668091C1
:103680008F05882309F450C018A219A21AA21BA200
:1036900020E030E040EA50E46091E4167091E516D5
:1036A0008091E6169091E7160E943AF369837A8337
:1036B0008B839C83BE01605E7F4FCE0101960E948A
:1036C000446D87EA9AE10E941D67809178128823F1
:1036D00019F081E08093771281E090E09093681276
:1036E00080936712109271121092721210927312DC
:1036F000109274120E944ABC60936D1270936E1205
:1037000080936F12909370128091670E9091680E63
:10371000A091690EB0916A0E8093691290936A121B
:10372000A0936B12B0936C128091DB168093F4051A
:103730000E94196C0E94C85D80912A1C982F9D7F61
:10374000943009F07FC090914017992309F478C014
:103750001092401710923C029091261C992351F12F
:10376000843069F460918E05862F90E0A0E0B0E08F
:10377000BC01CD01635E7F4F8E4F954A29C08630D4
:1037800009F05EC018A219A21AA21BA219821A82FD
:103790001B821C82BE01605E7F4FCE0101960E949B
:1037A000446D81E09AE590937E1580937D1586E1C6
:1037B00090E02EC0843099F460918E05862F90E0C1
:1037C000A0E0B0E0BC01CD01695B7F4F8E4F954A10
:1037D00024E830E040E050E00E94FA6631C08630D4
:1037E00079F518A219A21AA21BA219821A821B82A9
:1037F0001C82BE01605E7F4FCE0101960E94446D27
:1038000081E09AE590937E1580937D1580E490E0A9
:103810009093801580937F1587E08093711582E8DF
:103820008093741584E890E0A0E0B0E08093751573
:1038300090937615A0937715B09378150E945666ED
:1038400010922A1C20E030E040E251E46091DC1646
:103850007091DD168091DE169091DF160E9406EDC4
:103860000E947FF470937E1560937D1505E00093B0
:10387000711512E81093741588E490E1A0E0B0E0AF
:103880008093751590937615A0937715B09378155E
:103890000E94566620E030E040E251E46091E0167C
:1038A0007091E1168091E2169091E3160E9406ED68
:1038B0000E947FF470937E1560937D1500937115BF
:1038C000109374158AE490E1A0E0B0E08093751540
:1038D00090937615A0937715B09378150E9456664D
:1038E00020E030E040E251E46091E4167091E5168A
:1038F0008091E6169091E7160E9406ED0E947FF4F3
:1039000070937E1560937D15009371151093741557
:103910008CE490E1A0E0B0E080937515909376156B
:10392000A0937715B09378150E9456669091771200
:1039300080918F05992391F0811110C080914117DA
:1039400081110FC081E08093411780E493E0909350
:103950001511809314110E94C1D903C081111092D6
:103960008F0580912A1C813031F40E94716B109276
:103970002A1C0C94041280E00E94716B0C940412B7
:103980000E94EB560C940412C090DC16D090DD1609
:10399000E090DE16F090DF1688E50E94F7DA8111DC
:1039A00008C020E030E0A901C701B6010E943BF346
:1039B00002C00E9491DA68A379A38AA39BA3C09056
:1039C000E016D090E116E090E216F090E31689E55B
:1039D0000E94F7DA811108C020E030E0A901C70198
:1039E000B6010E943BF302C00E9491DA6B017C0198
:1039F00069837A838B839C832091EC163091ED163A
:103A00004091EE165091EF1668A179A18AA19BA171
:103A10000E943AF34B015C012FE632E143E85AEB96
:103A20000E9461F587FF02C00C94041221E230E08D
:103A300044EB53E4C501B4010E94A1EC181614F440
:103A40000C9404122091F0163091F1164091F21668
:103A50005091F316C701B6010E943AF36B017C0145
:103A60002FE632E143E85AEB0E9461F587FF02C07E
:103A70000C94041221E230E044EB53E4C701B60198
:103A80000E94A1EC181614F40C9404120C94BC2996
:103A900081E0809398050C94041285E40E94F7DA83
:103AA000B82E811102C00E9429CE75E6872E72E0E1
:103AB000972EECEDCE2EE6E1DE2EF4E8EF2EFAE1C5
:103AC000FF2E00E010E0A12C33243394D4018D911B
:103AD0004D010E94F7DA882359F1F60140805180A8
:103AE000628073800E9491DAD6016D937D938D93ED
:103AF0009C9313970330E1F0023011F43092F705F4
:103B0000A30192010E943AF39B01AC01F70160818D
:103B10007181828193810E943BF3D7016D937D93E4
:103B20008D939C931397C8010E94A36EAA24A3941B
:103B30000F5F1F4FB4E0CB0ED11CE4E0EE0EF11C82
:103B40000430110519F6AA2019F00E941ADA37C0BC
:103B5000BB20A9F1C090E816D090E916E090EA16D3
:103B6000F090EB162091BE163091BF164091C01612
:103B70005091C116C701B6010E9406ED0E946DF575
:103B80006093D3117093D4118093D5119093D61173
:103B9000C701B6010E947FF42FB7F8946093DB1B36
:103BA0007093DC1B8093DD1B9093DE1B2FBF109264
:103BB000C3111092C4111092C5111092C6110E9427
:103BC000C85D0C94041280916002882311F40C9457
:103BD000041289E40E94F7DA082F882321F00E945A
:103BE00061DA162F01C010E08AE40E94F7DAE82EAD
:103BF000882321F00E9461DAF62E01C0F12C002307
:103C000011F0143028F4EE2089F0F3E0FF1570F481
:103C1000E6E5F3E084918F010F5F1F4F882311F4D5
:103C20000C9404120E9414DBF801F4CF0E94276E5A
:103C3000002339F12091D7163091D8161203B00124
:103C4000139F700D11248091D3169091D416680F94
:103C5000791F072E000C880B990B0E94A7EC20916E
:103C6000EC163091ED164091EE165091EF160E9431
:103C70003BF36093931A7093941A8093951A9093E0
:103C8000961AEE2041F12091D9163091DA164F2D77
:103C90004203B001439F700D11248091D51690917D
:103CA000D616680F791F072E000C880B990B0E94FF
:103CB000A7EC2091F0163091F1164091F216509138
:103CC000F3160E943BF36093971A7093981A8093AF
:103CD000991A90939A1A80E50E94C8DA81110E947D
:103CE00082DA86E40E94F7DA8823D9F00E9491DA1A
:103CF0006B017C0120E030E0A9010E9461F51816FB
:103D000084F420E030E040E752E4C701B6010E94AD
:103D100017F46093340270933502809336029093C7
:103D200037020E9442AE0C94041280919905909142
:103D30009A058637910509F48EC60CF0C2C08D3401
:103D4000910509F4F1C30CF058C08A31910509F4CA
:103D500045C24CF58531910509F4E5C184F4823101
:103D6000910509F4A0C58431910509F49AC14197E0
:103D700011F00C9404120E94F1AD0C9404128731DE
:103D8000910509F4DCC10CF4D4C18831910509F422
:103D9000ECC1499711F00C940412109277120E9412
:103DA0007ACF0C9404128F31910509F4C7C274F4D0
:103DB0008C31910509F46EC20CF42FC24E9711F0AC
:103DC0000C9404120E94D8630C9404128A32910558
:103DD00009F467C32CF4809709F466C20C940412AA
:103DE0008B34910509F49CC38C34910511F00C942B
:103DF00004120E947ACF0C9404128A36910509F4B9
:103E000018C5BCF58435910509F44DC5ECF482352F
:103E1000910509F43FC50CF041C58135910511F0BC
:103E20000C9404120E9495C70E9429CE0E94E0AD16
:103E3000109245171092441768EE73E080E090E00E
:103E40000E94A0BC0C9404128C35910509F474C531
:103E500034F48535910509F454C50C940412883660
:103E6000910509F465C38936910509F495C40C944C
:103E700004128F36910509F497C384F48C369105AA
